:100000008A110A120528000009000730990083169A
:1000100005108510051185150516851283121430FB
:10002000AE000A30AF00051005112C30A0000130E1
:10003000A1008022851929281F308305051A292847
:100040002F080A3C031D2728AF01AE0172201F3084
:1000500083051F30830585193A281F308305051E47
:100060003A282F080A3C031D3828AF01AE0198201A
:100070001F3083051F308305851D4B281F308305E6
:10008000051A4B282E08143C031D4928AE01AF0168
:10009000D6201F3083051F308305851D5C281F3047
:1000A0008305051E5C282E08143C031D5A28AE014A
:1000B000AF0114211F3083051F308305E830A000F5
:1000C0000330A10080222E08013EAE002E083C3CE9
:1000D000031D6E282F08013EAF00AE011F308305BF
:1000E0001A28712805145830A0000230A10080227F
:1000F0007F212822A2212822D02128226321282200
:100100008E2136226A212822982136227F21282218
:100110005221282287212822A22128229C2136220E
:100120006E229030A0000130A1008022051008004E
:1001300005145830A0000230A1008022A6212822F8
:10014000A6212822A62136227F212822A221282288
:10015000D0212822632128228E2136227F212822A5
:10016000A2212822D0212822632128228E21362272
:100170007F212822A2212822D0212822632128227F
:100180008E2136226A21282265212822BE2128229A
:10019000DC2128229C2128226E2136226E229030DA
:1001A000A0000130A100802205100800051458307D
:1001B000A0000230A1008022A6212822A621282208
:1001C000A62136227F212822A2212822D0212822DE
:1001D000632128228E2128220F2228225F21362205
:1001E0007F212822A2212822D0212822632128220F
:1001F0008E2128220F2228225F2136227F212822C9
:10020000A2212822D0212822632128228E212822DF
:100210000F2228225F2136226E229030A00001306A
:10022000A10080220510080005145830A0000230FB
:10023000A1008022A6212822A6212822A62136223A
:100240007F212822A2212822E82128226321282296
:100250008A2128220F2228225F2136227F2128226C
:10026000A2212822E8212822632128228A2128226B
:100270000F2228225F2136227F212822A221282234
:10028000E8212822632128228A2128220F222822DD
:100290005F2136226E229030A0000130A100802222
:1002A000051008004C225D2208005D224C224C22E1
:1002B0004C2208005D224C225D224C2208005D2267
:1002C0004C224C2208004C2208004C224C225D2279
:1002D0004C2208005D225D224C2208004C224C2258
:1002E0004C224C2208004C224C2208004C225D2259
:1002F0005D225D2208005D224C225D2208004C2216
:100300005D224C224C2208005D225D2208005D2205
:100310004C2208005D225D225D2208004C225D22F5
:100320005D224C2208005D225D224C225D220800E5
:100330004C225D224C2208004C224C224C22080008
:100340005D2208004C224C225D2208004C224C22E7
:100350004C225D2208004C225D225D2208005D22B5
:100360004C224C225D2208005D224C225D225D223F
:1003700008005D225D224C224C2208005D225D2295
:100380005D225D225D2208004C225D225D225D22FD
:100390005D2208004C224C225D225D225D22080075
:1003A0004C224C224C225D225D2208004C224C2221
:1003B0004C224C225D2208004C224C224C224C2222
:1003C0004C2208005D224C224C224C224C22080078
:1003D0005D225D224C224C224C2208005D225D22CF
:1003E0005D224C224C2208005D225D225D225D22AE
:1003F0004C2208004C225D224C225D224C225D22C0
:1004000008005D225D224C224C225D225D22080004
:100410004C224C225D225D224C224C2208005D229F
:100420004C224C225D224C2208005D224C224C22A0
:100430004C225D2208005D224C224C224C224C2290
:100440005D22080005116430A000A101802208008F
:1004500005116430A000A10180226430A000A10138
:1004600080226430A000A1018022080005116430C0
:10047000A000A10180226430A000A101802264308C
:10048000A000A10180226430A000A101802264307C
:10049000A000A1018022080005150530840002306B
:1004A000AA009930A0000230A1004430A200003020
:1004B000A300BB2205112222080005150530840087
:1004C0000230AA009930A0000230A1000E30A20034
:1004D0000130A300BB2205112222080005150530BA
:1004E00084000230AA009930A0000230A100EE3052
:1004F000A2000230A300BB220511222208007F2A9D
:10050000A00803198B2A9222A0030000000000001B
:1005100000000000802AA108031908009222A1030C
:10052000A003802A0C30A500A50B942A000000002F
:100530001230A200A20BA12AA322A32200000000D5
:100540000800A3229A2A0D30A400A40BA52A0000BB
:1005500008001030A8020001031C013EA902031C80
:100560000800B22A0A30A8020001031C013EA902B9
:10057000031C0800B22A2A0880042008A8002108C9
:10058000A900A9220130A202031CA3032A098005A5
:100590002008A8002108A900A922A208031DBB2A3F
:0805A000A308031DBB2A08009B
:02400E00C431BB
:00000001FF
